:0614000002148B024A18E1
:01140B0032AE
:0114130032A6
:01141B00329E
:011423003296
:01142B00328E
:031433000242D49E
:01143B00327E
:011443003276
:03144B0002514308
:03145300021A95E5
:03145B00021D6F00
:011463003256
:03146B00024357E2
:011473003246
:01147B00323E
:03148300024D3CDB
:0314E90002148664
:03148600022E052E
:1014EC00AF83E58290F554F0EFA3F075E10490DF43
:1014FC003BE0FFBF01F890F554E0FEA3E0FF90DF66
:10150C0006EEF075E10290DF3BE0FFBF0DF8227EA6
:10151C00007F0090FC48E0FCA3E0FD8E028F03C32B
:10152C00EA9CEB9D503AEE2400FCEF34F0FD90FC6D
:10153C0046E0F514A3E0F5158A828B83C007C0063C
:10154C00C005C004125678AA82AB83D004D005D053
:10155C0006D0078C828D83EAF00EBE00B60F80B3E6
:10156C0022E58290F556F0E0FFE59CC39FF59CE5E3
:10157C009C24FAF59C439E10D2BA22AF9E74EF5F66
:10158C00F59E22AF83E58290F55AF0EFA3F090FC24
:10159C0041E0601390583A1243C690FC41E0F5824A
:1015AC001244087582EF2290FC417406F090DF3BE8
:1015BC00E0FFBF130280F6C29090F557E0FEA3E067
:1015CC00FF90FCA8EEF0EFA3F090FCA274F1F0E415
:1015DC00A3F090FC387472F074F3A3F090FCA0E4C8
:1015EC00F0A3F090FC53F090FC9CF090FC52F09027
:1015FC00FC9E04F0E4A3F090FC9D7402F090F55C6A
:10160C00E4F090000012173490F55AE0FEA3E0FFCE
:10161C0090F559E0FD7B007C008D017A00C3EB99BD
:10162C00EC9A50548B02EA75F0F0A42EF9E43FFAD0
:10163C0090F55C74F0F089828A83C007C006C005FF
:10164C00C004C003121734AA82D003D004D005D032
:10165C0006D007EA601B90588CC0021243C6D00219
:10166C0090FC41E4F08A82C002124408D0028A82C3
:10167C00220BBB00A40C80A190FCABE0FF30E33349
:10168C0090FCA8E0FEA3E0FFEE540F602690FCA8AF
:10169C00E0FEA3E053060F7F007410C39EFEE49F90
:1016AC00FF90FCA8E0FCA3E0FD90FCA8EE2CF0EF72
:1016BC003DA3F090FCA8E0FEA3E0FFC374FF9EE402
:1016CC009F502390FCA8E0FEA3E090DF02EEF09088
:1016DC00DF04E0FF74FC5FF0E0FF74024FF090FC5D
:1016EC00AA7401F0801290FCA8E0FEA3E0FF90DF4A
:1016FC0002EEF090FCAAE4F075E1037E607FEA90C4
:10170C00DF3BE0FDBD130280091EBEFF011FEE4F43
:10171C0070EDD290EE4F700C90FC667413F09058F4
:10172C00A41243C675820022AF83E58290F55DF06A
:10173C00EFA3F090F55CE0FF240F500A9058B5121F
:10174C0043C67582FF22EF703E90FC52E4F090FC91
:10175C0052E0FE90FC9DE0FDC3EE9D502190FC52AA
:10176C00E075F0F1A42472F58274F335F0F583E49E
:10177C00F090FC52E0FE0E90FC52EEF080D090FC0B
:10178C0052E4F07582002290FC41E0FE601DBE0622
:10179C001E90FC52E0601890DF3BE0FEBE1302800E
:1017AC000E90FC417407F07582ED227582ED22904B
:1017BC00FC52E075F0F1A42472FD74F335F0FE8D4B
:1017CC00828E83E0600A90FC667418F07582FE22AB
:1017DC008D828E8374FFF090FC52E075F0F1A4249E
:1017EC0072FD74F335F0FE0DBD00010E7C0090F51A
:1017FC005DE0FAA3E0FB8A148B158C168F037F0037
:10180C008B178F188D828E838CF0C007C0031255F6
:10181C009FD003D00790FCABE0FE20E3030218DC62
:10182C0090FC52E075F0F1A42472FD74F335F0FED7
:10183C000DBD00010E90FC7DEBF0EFA3F08D828EC0
:10184C00831252BDAE8290F55CEEF090FCABE0FFE3
:10185C00530704BF043F90FC52E075F0F1A42472CE
:10186C00FD74F335F0FF0DBD00010F8E037C00906D
:10187C00FCABE0FA5302F090FC81EDF0EFA3F0909A
:10188C00FC83EBF0ECA3F090FC85EAF08D828F8367
:10189C001252F7803B90FC52E075F0F1A42472FDDB
:1018AC0074F335F0FF0DBD00010F7C0090FCABE034
:1018BC00FB5303F090FC88EDF0EFA3F090FC8AEE64
:1018CC00F0ECA3F090FC8CEBF08D828F83125340E4
:1018DC0090FC52E075F0F1A42472FE74F335F0FF25
:1018EC0090F55CE0FD8E828F83F090FC52E0FF0F50
:1018FC0090FC52EFF090FC9DE0FEEFB5060590FCDD
:10190C0052E4F075820022AF83E58290F55FF0EF30
:10191C00A3F090FC41E0FF6014BF0102800F9058CF
:10192C00CF1243C690FC41E0F58212440812158791
:10193C0090FC4AE4F0A3F090FC4AE0FEA3E0FF8E9A
:10194C00828F83121A1590DF3BE0FFBF0DF890DFFA
:10195C003AE0FF53077FBF6000402790FC4AE0FE4F
:10196C00A3E0FF0EBE00010F90FC4AEEF0EFA3F0D7
:10197C00D29090000A124FC3C29090000A124FC32B
:10198C0080B590FC417402F090FC67E0FCA3E0FD94
:10199C00A3E0A3E090FC4CECF0EDA3F090F55FE03D
:1019AC00FEA3E0FF90FC50EEF0EFA3F02290FC4180
:1019BC00E4F090FC67E0FCA3E0FDA3E0A3E090FC66
:1019CC004CECF0EDA3F02290FC417404F090FC6719
:1019DC00E0FCA3E0FDA3E0A3E090FC4CECF0EDA355
:1019EC00F02290FC417405F090FC54E4F0A3F090CC
:1019FC00FC67E0FCA3E0FDA3E0A3E090FC4CECF062
:101A0C00EDA3F075820002156DAF83E58290F56150
:101A1C00F0EFA3F090F561E0FEA3E0FFEE2400F5FB
:101A2C0082EF34F0F583E0FF7E008F828E83021408
:101A3C00ECAF83E58290F563F0EFA3F090F563E0F3
:101A4C00FEA3E0FF90F370EEF0EFA3F0222290FCE7
:101A5C004AE0FEA3E0FF0EBE00010F90FC4AEEF040
:101A6C00EFA3F0C3EE9470EF9403400790FC4AE4AC
:101A7C00F0A3F090FC4AE0FEA3E0FFEE2400F58218
:101A8C00EF34F0F583E0F58222C021C0E0C0F0C055
:101A9C0082C083C007C006C005C004C003C002C01A
:101AAC0001C000C0D075D00090FC3DE02401F0A333
:101ABC00E03400F090FC42E0FEA3E0FF90FC3DE03F
:101ACC00FCA3E0FDECB5060BEDB5070790FC3DE47F
:101ADC00F0A3F090FC3DE0FEA3E0FFBE0005BF00CC
:101AEC0002800BBE0105BF00028068021C5790FCEF
:101AFC003DE0FEA3E08E077E00AC9C7D00EC420630
:101B0C00ED420790FC4EEEF0EFA3F090FC4AE0FEA5
:101B1C00A3E0FF0EBE00010F90FC4AEEF0EFA3F025
:101B2C0090FC48E0FCA3E0FDC3EE9CEF9D400790C9
:101B3C00FC4AE4F0A3F090DF3BE0FFBF1303021D6F
:101B4C005290FC4AE0FEA3E0FF8E828F83121A159E
:101B5C00021D5290FC41E0FFBF05028003021D52A2
:101B6C00900019124FC390F567741CF090FC4AE07A
:101B7C00FEA3E090F568EEF090FC4AE0A3E090F54F
:101B8C0069F090F56A7442F090F56B744CF090F536
:101B9C006C7441F090F56D7448F090F56E7442F0F1
:101BAC0090F56F744CF090F5707441F090F5717481
:101BBC0048F090F5727442F090F573744CF090F517
:101BCC00747441F090F5757448F090F5767442F0A9
:101BDC0090F577744CF090F5787441F090F5797439
:101BEC0048F090F57A7442F090F57B744CF090F5D7
:101BFC007C7441F090F57D7448F090F57E7442F061
:101C0C0090F57F744CF090F5807441F090F58174F0
:101C1C0048F090F5827420F090FC56741CF0E4A30C
:101C2C00F090FC58F0A3F090FC5AF0A3F090F568FB
:101C3C0012469190FC54E0FEA3E0FF0EBE00010F93
:101C4C0090FC54EEF0EFA3F0021D5290FC41E0FF2B
:101C5C00BF03028065BF04028008BF050280030237
:101C6C001D5290FC4CE0FEA3E0FF90FC67E0FAA351
:101C7C00E0FBA3E0FCA3E0FD8E008F01E4FEFFEA95
:101C8C00C398FAEB99FBEC9EFCED9FFDC374649A30
:101C9C00E49BE49CE49D50229058FD1243C690FCBA
:101CAC00417405F090FC67E0FCA3E0FDA3E0FEA30B
:101CBC00E0FF90FC4CECF0EDA3F090FC53E075F0E1
:101CCC00F1A42472FE74F335F0FF8E828F83E060F2
:101CDC0075900019124FC390FC53E075F0F1A424D9
:101CEC0072FE74F335F0FF90DF04E05401FDB40193
:101CFC0000E4332EFDE43FFC8E828F83E090FC5693
:101D0C00F0E4A3F090FC58F0A3F090FC5AF0A3F090
:101D1C008D828C8312469190FC53E075F0F1A424D3
:101D2C0072F58274F335F0F583E4F090FC53E0FF28
:101D3C000F90FC53EFF0BF0200400590FC53E4F011
:101D4C0090591B1243C6D0D0D000D001D002D00382
:101D5C00D004D005D006D007D083D082D0F0D0E00C
:101D6C00D021323290FC41E4F090FC52F090FC53C4
:101D7C00F090FC4AF0A3F090FC467453F0E4A3F00E
:101D8C0090FC487453F0E4A3F090FC4EF0A3F09058
:101D9C00FC4CF0A3F090FC427406F0E4A3F090FC31
:101DAC0044F0A3F090FC50F0A3F090FC54F0A3F09E
:101DBC0012151B90FC41E4F0759DDC859E9E439EA4
:101DCC000443CB1022021D709021F812334D90FC6D
:101DDC0067E4F0A3F0A3F0A3F0121DD190F583E417
:101DEC00F090F5847432F074F8A3F02290FC41E08A
:101DFC00FFBF000302212DBF0103021FFEBF020320
:101E0C00021EFCBF030302212DBF040302212DBFC0
:101E1C00050302210EBF060122BF40028006BF410E
:101E2C000280422275E10490DF3BE0FFBF01F89095
:101E3C00DF0374E5F090DF047404F090DF07741294
:101E4C00F090DF08E4F090DF147410F090DF17E0EE
:101E5C00FF74C04FF090FC417441F090F5847432E3
:101E6C00F074F8A3F090F583E4F090FC54E0FEA33A
:101E7C00E0FF90F583E0FDFB7C00C3EB9EEC9F50F4
:101E8C004590DF06EDF075E10490DF3BE0FFBF010C
:101E9C00F875E10290DF3BE0FFBF0DF890000212F5
:101EAC004FC390F584E0FEA3E0FF90F583E02EFE97
:101EBC00E43FFF90DF3AE0FD8E828F83F090F58354
:101ECC00E02401F080A475E10490DF3BE0FFBF014A
:101EDC00F890FC54E0FEA3E08E3375340090F5844A
:101EEC00E0F535A3E0F536753201758243022E37E5
:101EFC00E50F7003021FEC90FC65740DF0AF9A7443
:101F0C00FE5FF59AE50F20E403021FEC90FC417490
:101F1C0003F090FC3FE0FEA3E08E8212156D905909
:101F2C00291243C690FC3FE0FEA3E0FF8E828F8314
:101F3C0012442390F831E025E0FEE42432FFEE3425
:101F4C00F8FE8F828E831243C690F831E0FFB40105
:101F5C0000E433FF90F583F0EF2436FDE434FCFE0F
:101F6C008D828E83E0707290DF04E0FE30E0378F5C
:101F7C0006EE2EFDE42432F582ED34F8F583E0FE16
:101F8C008E337534008F06EE2EFDE42432FEED34D4
:101F9C00F8FD74012EF535E43DF536753201758288
:101FAC0042122E37802290DF02E0FE8E33E4F534AD
:101FBC00EF2FFEE42432FFEE34F8FE8F358E3675AB
:101FCC003201758242122E3790F583E0FF2436F5EC
:101FDC0082E434FCF5837401F0AF0F74EF5FF50FFE
:101FEC00D20010AF02C200750F00A20092AF439A4C
:101FFC000122E50F70030220FC90FC65740DF0AF1C
:10200C009A74FE5FF59AE50F20E4030220FC90F829
:10201C0031E0FF90F583B40100E433F090593E12A7
:10202C0043C690F583E025E0FEE42432FFEE34F85D
:10203C00FE8F828E8312442390F583E025E0FEE42C
:10204C002432FFEE34F8FE8F828E831243C690F852
:10205C0031E0FFB40100E433FF90F583F0EF243658
:10206C00FDE434FCFE8D828E83E0707290DF04E020
:10207C00FE30E0378F06EE2EFDE42432F582ED348F
:10208C00F8F583E0FE8E337534008F06EE2EFDE4FA
:10209C002432FEED34F8FD74012EF535E43DF536B1
:1020AC00753201758242122E37802290DF02E0FEDB
:1020BC008E33E4F534EF2FFEE42432FFEE34F8FED9
:1020CC008F358E36753201758242122E3790F5831C
:1020DC00E0FF2436F582E434FCF5837401F0D20081
:1020EC0010AF02C200AF0F74EF5FF50FA20092AFFA
:1020FC00D20010AF02C200750F00A20092AF439A3B
:10210C00012290FC54E0FEA3E0FF90FC48E0FCA30D
:10211C00E0FDC3EE9CEF9D50012290FC417404F055
:10212C0022E50F70012290FC65740DF0E50F543020
:10213C0070012290F831E0FFB40100E433FF90F518
:10214C0083F0EF2436FDE434FCFE8D828E83E06058
:10215C00030221E590DF04E0FE30E0378F06EE2E1F
:10216C00FDE42432F582ED34F8F583E0FE8E337510
:10217C0034008F06EE2EFDE42432FEED34F8FD74AF
:10218C00012EF535E43DF536753201758242122E7D
:10219C0037803590FC97E0E0600A90FC9AE0FDA354
:1021AC00E0FE800890DF02E0FCFD7E00EF2FFCE4F7
:1021BC002432FFEC34F8FC8F358C367532018D33BC
:1021CC008E34758242122E3790F583E0FF2436F55B
:1021DC0082E434FCF5837401F0D20010AF02C2002B
:1021EC00AF0F74CF5FF50FA20092AF2290F7E3E030
:1021FC00FDA3E0FEA3E0FF90F7E8E0FCBC42028008
:10220C0003022B9390F7E9E0FC24BE5003022B85CC
:10221C00EC240A83F582EC244683F583E4738585EC
:10222C00FE4685B16C8A9DD60F3376148585DA59B6
:10223C0080F3182B970B4085858585858585EA73FA
:10224C00BAB0D38585858585858585858585858584
:10225C008585858585858585858585858585AEE896
:10226C002B2B22252B2324242424252525262B2BFC
:10227C00282929292A2A2A28292B2B2B2B2B2B2BB3
:10228C002A2B2A29292B2B2B2B2B2B2B2B2B2B2B98
:10229C002B2B2B2B2B2B2B2B2B2B2B2B2B2B2B2B82
:1022AC002222C007C006C005121587D005D006D063
:1022BC000790FC417440F08D828E838FF01257D7BB
:1022CC00FC7B0090FC54ECF0EBA3F090F809EDF0E3
:1022DC00EEA3F0758201124118022B9390FC41E49D
:1022EC00F090F809EDF0EEA3F0758201124118029E
:1022FC002B9390FC41E060099059581243C6022B75
:10230C00938D828E838FF01257D7FC7B0090F586CD
:10231C00ECF0EBA3F08D828E83A3E0FAE4F92CFCB5
:10232C00EA3BFB90F586ECF0EBA3F08D828E83A359
:10233C00A3A3A3E0FA8A0889098D828E83A3A3A3A1
:10234C00A3A3E0FAE42508F508EA3509F50990FCA1
:10235C003AE4F0A3F074062DF9E43EFA90FC56EC46
:10236C00F0EBA3F090FC58E4F0A3F090FC5AE508D5
:10237C00F0E509A3F089828A83C007C006C0051264
:10238C004691AC82D005D006D0078D828E838FF01B
:10239C00EC12564090F809EDF0EEA3F075820112A4
:1023AC004118022B938D828E838FF01257D790FC9D
:1023BC009AF0E4A3F08D828E83A3E0FB7C0090FC6A
:1023CC009AE0F9A3E0FA90FC9AEC29F0EB3AA3F02E
:1023DC0090FC9AE0A3E090FC9AE0F5F0A3E045F0C5
:1023EC00604B90FC977401F090FC98E0A3E090FC9B
:1023FC0098E0F5F0A3E045F070471245CA90FC9ABE
:10240C00E0FBA3E0FC90FC98EBF0ECA3F090FC98C4
:10241C00E0FBA3E090DF02EBF090DF04E0FC74FC47
:10242C005CF0E0FC74024CF0124580801490FC9738
:10243C00E4F090FC98F0A3F090FC9AF0A3F0124515
:10244C00CA90F7E8E0FC90F7E9E0F53275359A753B
:10245C0036FC7533017534008C82122E37022B93A7
:10246C008D828E838FF01257D790FCABF090F809C9
:10247C00EDF0EEA3F0758201124118022B9390F847
:10248C000974ABF074FCA3F0758201124118022B95
:10249C009390FCABE0FC5304F090FC797406F09044
:1024AC00FC7AECF08D828E838FF0C007C006C005DD
:1024BC00125265D005D006D00790F809EDF0EEA3C6
:1024CC00F0758210124118022B9390FCABE0FC5378
:1024DC0004F090FC797404F090FC7AECF08D828E10
:1024EC00838FF0C007C006C005125265D005D00618
:1024FC00D00790F809EDF0EEA3F075821012411898
:10250C00022B938D828E838FF01257D790FCACF0F8
:10251C00E0FC74015CF090F809EDF0EEA3F075822C
:10252C0001124118022B9390F80974ACF074FCA3BF
:10253C00F0758201124118022B938D828E838FF0DD
:10254C001257D7FC7B008C828B83C007C006C0055A
:10255C00121A3DD005D006D00790F809EDF0EEA385
:10256C00F0758201124118022B9390FC41E0601C23
:10257C008D828E838FF074EF12564090F809EDF037
:10258C00EEA3F0758201124118022B938D828E837B
:10259C008FF01257D7FC7B0090F586ECF0EBA3F094
:1025AC008D828E83A3E0FAE42CFCEA3BFB90F5864B
:1025BC00ECF0EBA3F08D828E83A3A3E0FA90FC3AAF
:1025CC00E4F0A3F074032DF8E43EF990F557ECF029
:1025DC00EBA3F090F559EAF088828983C007C00616
:1025EC00C00512158FAC82D005D006D0078D828E17
:1025FC00838FF0EC12564090F809EDF0EEA3F075D5
:10260C008201124118022B938D828E838FF0125708
:10261C00D7FB7C0090F586EBF0ECA3F0EB4C600361
:10262C0002271C90FCA8E0A3E090FCA8E0F5F0A326
:10263C00E045F0601C90DF3BE0FABA1314900028E0
:10264C00C007C006C005124FC3D005D006D0078006
:10265C00D290FCA8E0A3E090FCA8E0F5F0A3E04544
:10266C00F0606B90597DC007C006C0051243C69040
:10267C00FCA8E0F9A3E0FA89828A8312442390F340
:10268C0072E0F58212440890F463E0F5821244087B
:10269C00D005D006D00790FC667412F08D828E8324
:1026AC008FF074EC125640C290C007C006C00512E1
:1026BC00455BD005D006D00790FC41E4F090F809BA
:1026CC00EDF0EEA3F0758201124118022B93C2902B
:1026DC0090FC41E4F08D828E838FF012564090591D
:1026EC0091C007C006C0051243C690FC3AE0F9A39E
:1026FC00E0FA89828A83124423D005D006D0079051
:10270C00F809EDF0EEA3F0758201124118022B933B
:10271C0090FC41E0FABA060280619059A1C007C052
:10272C0006C0051243C6D005D006D00790FC66E063
:10273C00FABA121B8D828E838FF074EC1256409075
:10274C00F809EDF0EEA3F0758201124118801F908C
:10275C00FC667417F08D828E838FF074EF125640E6
:10276C0090F809EDF0EEA3F0758201124118C290B9
:10277C0012455B90FC41E4F0022B9374012DF9E4BB
:10278C003EFA90F55CEBF089828A83C007C006C0E4
:10279C0005121734AC82D005D006D0078D828E83FB
:1027AC008FF0EC1256408D828E838FF01257D7FB30
:1027BC00EC603BBBFE0280369059AAC007C006C035
:1027CC00051243C6D005D006D0078D828E838FF0BC
:1027DC001257D7F582C007C006C005124408C29034
:1027EC0012455BD005D006D00790FC41E4F090F880
:1027FC0009EDF0EEA3F0758201124118022B938DB6
:10280C00828E838FF01257D7FB7C0090F586EBF00D
:10281C00ECA3F0C374F09BE49C50199058B5124390
:10282C00C690F8097486F074F5A3F0758201124114
:10283C0018022B9390FC52E075F0F1A42472F974F9
:10284C00F335F0FA89828A83E060199059B7124304
:10285C00C690F8097486F074F5A3F07582011241E4
:10286C0018022B938B0089828A83E8F090FC52E04B
:10287C0075F0F1A42472F974F335F0FA09B900017A
:10288C000A890A8A0B750C0074012DF9E43EFA8949
:10289C00148A157516008B178C18850A82850B8384
:1028AC00850CF012559F90FC52E0FC0C90FC52EC05
:1028BC00F0BC0200400590FC52E4F090F8097486DC
:1028CC00F074F5A3F0758201124118022B938D82DE
:1028DC008E838FF01257D7FC7B0090FC46ECF0EB0C
:1028EC00A3F090FC46E0F9A3E0FAC374709C740367
:1028FC009B402E74022DFBE43EFC8B148C1575163C
:10290C000089178A1890F00075F00012559F90F806
:10291C00097446F074FCA3F0758202124118022B64
:10292C009390F80974D8F07459A3F0758208124189
:10293C0018022B9390FC46E0FBA3E090F80974007E
:10294C00F074F0A3F08B82124118022B93121A5AD6
:10295C007B008B83121A1590FC4AE0FBA3E0FC90E1
:10296C00F809EB2400F0EC34F0A3F075820112416D
:10297C0018022B938D828E838FF01257D7FC7B001D
:10298C008C828B83C007C006C0051214ECD005D016
:10299C0006D00790F809EDF0EEA3F0758201124114
:1029AC0018022B93758200C007C006C00512156D66
:1029BC00D005D006D00790F809EDF0EEA3F07582A3
:1029CC0001124118022B93C007C006C005121587CF
:1029DC00D005D006D00790F809EDF0EEA3F0758283
:1029EC0001124118022B938D828E838FF01257D7D0
:1029FC00FC7B0090FC42ECF0EBA3F090F809EDF0BE
:102A0C00EEA3F0758201124118022B9390F8097411
:102A1C0042F074FCA3F0758204124118022B938DC2
:102A2C00828E838FF0C007C006C005124385D00587
:102A3C00D006D0078D828E838FF01257D7F582C0C7
:102A4C0007C006C005124408D005D006D0078D82F9
:102A5C008E838FF01257D7FC7B008C148B158B1642
:102A6C007517158B1890FC4175F000C007C006C097
:102A7C000512559FD005D006D00790F809EDF0EE61
:102A8C00A3F0758215124118022B9390FC3DE0FBCC
:102A9C00A3E0FC90FC44EBF0ECA3F090F80974413B
:102AAC00F074FCA3F0758215124118022B938D82E1
:102ABC008E838FF01257D7FC7B008C828B83C007E0
:102ACC00C006C005121913D005D006D00790F8091E
:102ADC00EDF0EEA3F0758201124118022B9390FCDD
:102AEC0067E0F9A3E0FAA3E0A3E090FC4CE9F0EA7C
:102AFC00A3F08D828E838FF01257D7FC90FC41F09F
:102B0C0090FC41E0FBEC24FA404DEB2B2B902B1D61
:102B1C0073022B2F022B2F022B2F022B51022B5126
:102B2C00022B40C007C006C005121587D005D00681
:102B3C00D0078023C007C006C0051219EED005D0FF
:102B4C0006D0078012758200C007C006C00512159A
:102B5C006DD005D006D00790F809EDF0EEA3F07516
:102B6C008201124118802090F8097441F074FCA382
:102B7C00F0758201124118800E90F809EDF0EEA369
:102B8C00F0758201124118900000222290F7F1E0BA
:102B9C00FFBF013990F7D1E0FEA3E0FF90F7F4E01E
:102BAC00FCA3E0FD90F7D4E0FAA3E0FBEA4B601D38
:102BBC008E828F83E0F9A3AE82AF838C828D83E902
:102BCC00F0A3AC82AD831ABAFF011B80DF90F7DA59
:102BDC00E054FDF090DE11E0FF74084FF022AE825D
:102BEC00AF83E0FD20E703022CE38E828F83A3E00A
:102BFC00FD601DBD0102802ABD0202803BBD0302A7
:102C0C00805ABD04028076BDFE03022CA5022CE383
:102C1C0075370275380090FC6575F0001230E502CE
:102C2C002CE390DE00E0FD7C007539288C3A8D8217
:102C3C008C83123159022CE38E828F83A3A3E0FC88
:102C4C00A3E0FD74062EF582E43FF583E0F539A38D
:102C5C00E0F53A8C828D83123159807B8E048F057E
:102C6C007B0074062EF582E43FF583E0F537A3E094
:102C7C00F5388C828D838BF01230E5805A90F7D129
:102C8C00E0FBA3E0FCA3E0FD753910753A008B82E4
:102C9C008C838DF0123159803E74022EFEE43FFF7E
:102CAC007D00756BE0756C59756D807514048D1510
:102CBC008E828F838DF012508FE5828583F045F0E4
:102CCC006012D29090012C124FC3C29090012C1222
:102CDC004FC3800375C9839000002290DF2FE4F06E
:102CEC0090DF30F090DF31F090DF00740CF090DF6B
:102CFC0001744EF090DF0274FFF090DF037440F02B
:102D0C0090DF04E4F090DF05F090DF06F090DF0731
:102D1C007406F090DF08E4F090DF097424F090DF83
:102D2C000A743AF090DF0B74F1F090DF0C74CAF077
:102D3C0090DF0D74A3F090DF0E7401F090DF0F7430
:102D4C0023F090DF107411F090DF117436F090DFE7
:102D5C00127407F090DF13740FF090DF147418F0F6
:102D6C0090DF1514F090DF16746CF090DF1774037D
:102D7C00F090DF187440F090DF197491F090DF1A26
:102D8C007456F090DF1B7410F090DF1C74E9F09017
:102D9C00DF1D742AF090DF1EE4F090DF1F741FF02B
:102DAC0090DF237488F090DF247431F090DF257469
:102DBC0009F090DF2E74C0F090DF07C4F090DF09AB
:102DCC007425F090DF0A7495F090DF0B7455F09039
:102DDC00DF1A74B6F090DF1B7410F090DF1C74EAED
:102DEC00F090DF1D742AF090DF1EE4F090DF1F746A
:102DFC001FF02212511102513D122DFF12446D127F
:102E0C00516A1230B0124603121DD41230DFD2AF09
:102E1C00122F82D290900002124FC3C29090000ADF
:0B2E2C00124FC3124149121DF880F83C
:10583A0043616E6E6F742063616C6C207472616E6A
:10584A00736D69745F6C6F6E67207768696C652029
:10585A004648535320486F7070696E67206F7220F4
:10586A00616C72656164792070726F6365737369C4
:10587A006E67207472616E736D69745F6C6F6E67A8
:10588A0021004D41435F747828292072657475722E
:10589A006E6564206572726F72006E65766572203D
:1058AA00656E74657265642054580046485353788F
:1058BA006D6974206D65737361676520746F6F20FD
:1058CA006C6F6E6700464853532073746174652089
:1058DA00656E746572696E672053594E4348494E26
:1058EA00472066726F6D2077726F6E6720737461DE
:1058FA0074650053594E43485F4D415354455220F5
:10590A002D3E2053594E43494E474D41535445521B
:10591A000046485353786D697420646F6E65006E53
:10592A006574776F726B207061636B657428737925
:10593A006E6329006E6574776F726B207061636B9A
:10594A00657428646973636F766572792900637276
:10595A0061702C20706C65617365207573652046D3
:10596A00485353786D6974282920696E7374656188
:10597A0064210064726F706F75742066696E616C61
:10598A0020776169742100746F74616C2062797484
:10599A0065732074783A00756E64657272756E006C
:1059AA00627566666572206572726F7200737469D9
:1059BA006C6C2077616974696E67206F6E207468F9
:1059CA0065206C617374207061636B6574004E4F5F
:0B59DA00204445414C005253544E0045
:102E3700AF827E0190DE0E7405F090FC657412F08F
:102E4700E53345347003022F787C107D2790DE111F
:102E5700E0FB30E00D90FC667401F01CBCFF011D27
:102E670080EBEC4D7014D2909003E8124FC3C290E0
:102E77009003E8124FC390FFFF22BE012C7E009003
:102E8700DE2A7440F0EFF0E532F0AC337D00ECF071
:102E9700E534F0C3743B9533E4953450067C3B7DB1
:102EA70000801AAC33AD348014C374409533E49575
:102EB7003450067C407D008004AC33AD34748025EB
:102EC7002942D6852682852783AA35AB368B01E929
:102ED700F0852682852783A3EAF0852682852783C6
:102EE700A3A374DEF0852682852783A3A3A3742A70
:102EF700F0852682852783A3A3A3A3A3ECFBF085F4
:102F07002682852783A3A3A3A3E054E0F085268226
:102F1700852783A3A3A3A3A3A3A3E0543F4440F01F
:102F2700852682852783A3A3A3A3A3A3A3E054CFC6
:102F3700F0E52942D6E52942D7E52955D160FAE5DA
:102F470029F452D190DE0E7405F090DE11E0FB7487
:102F5700014BF0E533C39CF533E5349DF534EC259F
:102F670035F535ED3536F53690FC657413F0022EE0
:102F77004790FC657414F090000022E5227005125A
:102F8700414980F722AFBE747F5FF5BE43BE809094
:102F9700DE0B7407F090DE077411F090DE0914F071
:102FA700438C10AF8C74FE5FF58CD2BD439A0275CB
:102FB7008900C2C5758B00C2E843A90243B90285DF
:102FC7002682852783A3A3A3A3E054E0F085268266
:102FD700852783A3A3A3A3A3A3E0549F4420F0853D
:102FE7002682852783A3A3A3A3A3A3A3E04408F072
:102FF700852682852783A3A3A3A3A3A3A3E054FCC9
:103007004401F090DE01E0FF74FE5FF0E4F525F582
:1030170023F524F52290DE0EF090DE107408F09070
:10302700DE13F090F7DBE4F090F7DAF090F7CFF0EB
:10303700A3F090F7D17488F074F5A3F0E4A3F090AF
:10304700F7D4F0A3F090F7D6F090F7D7F090F7D831
:10305700F0A3F090DE0E7405F090DE107408F09087
:10306700DE13F090DE12E0FF74014FF090DE15E002
:10307700FF74014FF090F7EDE4F090F7ECF090F764
:10308700E1F0A3F090F7E374C8F074F5A3F0E4A3BC
:10309700F090F7E6F0A3F090F7E8F090F7E9F090FA
:1030A700F7EAF0A3F0439A02221244978582288513
:1030B70028F005F07401800225E0D5F0FBF529E53D
:1030C7002875F008A42419F52674F835F0F527902B
:1030D700FC657402F0022F8CD29122C29122AFF0CC
:1030E700AE83E58290F7F6F0EEA3F0EFA3F090F74A
:1030F700DBE06034D2909003E8124FC3C290900394
:10310700E8124FC3D2909003E8124FC3C2909003C6
:10311700E8124FC3D2909003E8124FC3C2909003B6
:10312700E8124FC390FFFF2290F7F6E0FDA3E0FE01
:10313700A3E0FF90F7CCEDF0EEA3F0EFA3F090F74C
:10314700CFE537F0E538A3F090F7DB7401F0900096
:103157000022AF83E58290F7F9F0EFA3F090F7DB59
:10316700E06034D2909003E8124FC3C2909003E816
:10317700124FC3D2909003E8124FC3C2909003E856
:10318700124FC3D2909003E8124FC3C2909003E846
:10319700124FC390FFFF2290F7F9E0FEA3E0FF7DF7
:1031A7000090F7CCEEF0EFA3F0EDA3F090F7CFE5AA
:1031B70039F0E53AA3F090F7DB7401F090000022B4
:1031C7007F0290DE0EE4F090F7CFE0FDA3E0FEC3B0
:1031D70074409DE49E50047C4080048D047F0A8CDB
:1031E700027B00EDC39AFDEE9BFE90F7CFEDF0EE6C
:1031F700A3F08C06EE603690F7CCE0FBA3E0FCA3CF
:10320700E0FD8B828C838DF01257D790DE20F090F3
:10321700F7CCE0FBA3E0FCA3E0FD0BBB00010C90A7
:10322700F7CCEBF0ECA3F0EDA3F01E80C790DE1116
:10323700E04FF090F7CFE0FEA3E0FF4E700590F768
:10324700DBE4F02290F7DB7402F07582002290F73E
:10325700D1E0FDA3E0FEA3E0FF90DE11E0FCB401A6
:1032670000E433FC20E0F290DE0EE4F090DE16E09E
:10327700FC7B0090F7D4ECF0EBA3F090F7DAE0FCDE
:1032870030E11390F7DB7403F090DE11E0FC740477
:103297004CF090FFFF2290F7DAE04402F090F7D469
:1032A700E0FBA3E0FCC374409BE49C501CD29090CD
:1032B700012CC007C006C005124FC3C29090012C55
:1032C700124FC3D005D006D00790F7D4E0FBA3E098
:1032D700FC8D07EB4C601690DE20E0FD8F828E831D
:1032E700F0A3AF82AE831BBBFF011C80E6E52C4534
:1032F7002D6009852C82852D8312148990F7D4E0DF
:10330700FEA3E0FFC3EE9440EF9400501DE52A456D
:103317002B6009852A82852B8312148990DE11E0A0
:10332700FF74084FF090F7DBE4F090DE11E0FF74D4
:10333700404FF090F7D4E0FEA3E08E82F58322851C
:10334700822E85832F22858230858331227537012E
:1033570075380090002575F0400230E5AFF0AE8378
:10336700E58290F7FBF0EEA3F0EFA3F090F7FBE018
:10337700FDA3E0FEA3E0FF74022DFDE43EFE8D8277
:103387008E838FF01257D7FDA31257D78D2575223D
:103397000122AF827D1E7E5A8D828E83A3E090F735
:1033A700FEF09013E0E0F9A3E0FAA3E0FBA3E0FC52
:1033B700E4B9400ABA6C07BB6104BC730104FCE4BE
:1033C700BF030104FBAA1490F7FEE0F9B9FF0280DE
:1033D7004DE9B50732EB600CBA0309EC60067DE4F2
:1033E7007E13803AEA700890F7FE74FFF080D81ACF
:1033F7008D828E83E02DFDE43EFE8D828E83A3E0D9
:10340700F990F7FEF080C08D828E83E02DFDE43EBB
:10341700FE8D828E83A3E0F990F7FEF080A98D825E
:103427008E8322AFF0AE83E58290F7FFF0EEA3F034
:10343700EFA3F090F7FFE0F53DA3E0F53EA3E0F53D
:103447003F7402253DFAE4353EFBAC3F8A828B830D
:103457008CF01257D7F8A31257D7F9893B753C0060
:103467007402B53B06E4B53C0280227407B53B06FF
:10347700E4B53C028002804274AF58FE7F008A8226
:103487008B838CF0EE125640A3EF1256408A828B44
:10349700838CF01257D7FAA31257D7F5828A1412E2
:1034A7003399AE82AF8390F802EEF0EFA3F08E82ED
:1034B7008F83A3A3E0FE7F00801C898288141233C8
:1034C70099AC82AD8390F802ECF0EDA3F08C828D7D
:1034D70083E0FCFE7F007406253DFBE4353EFCAD32
:1034E7003F8B828C838DF01257D7FCA31257D7FDE1
:1034F700C3EC9EED9F50048C068D07EE4F7009902C
:10350700DE11E0FD74204DF090F802E0FCA3E0FD31
:103517008E398F3A8C828D8302315990DE0EE4F01A
:1035270090DE11E0FF30E40E90F7DBE4F090DE115F
:10353700E0FE74804EF0EF30E22490DE11E4F0906C
:10354700FC667404F090F7DBE4F0D290900014C0AE
:1035570007124FC3C290900014124FC3D00790F7C1
:10356700DBE0FEBE0319D290900032C007124FC3B2
:10357700C290900032124FC3D00790F7DBE4F0906F
:10358700F7DBE06003023862EF20E0030238629065
:10359700DE0EE4F090DE16E0FFFE7B407C007D400F
:1035A700EE601690DE20E0FA8B828C838DF0125647
:1035B70040A3AB82AC831E80E7E540FE20E7030211
:1035C700373574605EFD6015BD20030236EFBD40E0
:1035D700030236FBBD600302372002384A741F5EC0
:1035E700FF7041AD41BD0002801CBD06028005BDD4
:1035F7000826800C90004075F04012342A02384AA1
:1036070012335402384A7537027538009059FC75E1
:10361700F0801230E502384A90004075F0401243BE
:103627008402384ABF0145AD41BD00028005BD0A8D
:103637002680127537027538009059FC75F0801294
:1036470030E502384A7537017538009059FF75F033
:10365700801230E502384A90DE11E0FD74204DF00B
:1036670090004075F04012438402384ABF0236ADDD
:1036770041BD00028008BD120302384A8012753727
:10368700027538009059FC75F0801230E502384A0F
:1036970090DE11E0FD74204DF090004075F040126F
:1036A700438402384ABF032BE4B5411275370275CC
:1036B70038009059FC75F0801230E502384A90DEE8
:1036C70011E0FD74204DF090004075F040124384E6
:1036D70002384A90004075F04012438490DE11E0B2
:1036E700FD74204DF002384A90DE11E0FD74204D44
:1036F700F002384AE52E452F6013123706800BC0BB
:103707002EC02F90004075F0402202384A900040AA
:1037170075F04012387902384A90DE11E0FD7420C6
:103727004DF090004075F04012438402384A7460AF
:103737005EFD6015BD2003023801BD400302381548
:10374700BD600302383802384A741F5EFF7048AE06
:1037570041BE010302384ABE030302384ABE0502CE
:10376700800BBE070302384ABE0917800990DE00A6
:10377700E542F002384A90004075F0401233630288
:10378700384A90004075F04012438490DE11E0FE05
:1037970074204EF002384ABF0129AE41BE01030230
:1037A700384ABE030302384ABE110302384A900062
:1037B7004075F04012438490DE11E0FE74204EF015
:1037C70002384ABF0220AF41BF01028076BF030221
:1037D700807190004075F04012438490DE11E0FF45
:1037E70074204FF0805D90DE11E0FF74204FF09061
:1037F700004075F040124384804990004075F040C6
:1038070012438490DE11E0FF74204FF08035E52EDF
:10381700452F6012123820800BC02EC02F90004019
:1038270075F04022801D90004075F0401238798075
:103837001290DE11E0FF74204FF090004075F040C9
:1038470012438490DE11E0FF74404FF0E546454790
:10385700700990DE11E0FF74084FF090F7DBE0FF8E
:10386700BF01031231C790F7DBE0FFBF020302324B
:103877005522AFF0AE83E58290F804F0EEA3F0EFA7
:10388700A3F090F804E0FDA3E0FEA3E0FF8D828E95
:10389700838FF01257D7FC20E7030239D374012D29
:1038A700FAE43EFB8F048A828B838CF01257D7FC95
:1038B700601EBC0102802BBC0202803CBC0302805C
:1038C70073BC0403023970BCFE0302398D023A3916
:1038D70075370275380090FC6575F0001230E50207
:1038E7003A3990DE00E0FC7B007539288B3A8C82F0
:1038F7008B83123159023A3974022DFAE43EFB8F59
:10390700048A828B838CF01257D7FAA31257D7FBFE
:1039170074062DF8E43EF98F04888289838CF012AF
:1039270057D7F539A31257D7F53A8A828B831231C5
:1039370059023A398D028E038F048A488B498C4A83
:1039470074062DF8E43EF98F04888289838CF0127F
:1039570057D7F537A31257D7F53885488285498356
:10396700854AF01230E5023A3990F7D1E0FAA3E040
:10397700FBA3E0FC753910753A008A828B838CF0C3
:10398700123159023A3974022DFAE43EFB8F049042
:10399700FC6B7401F0745AA3F07480A3F0751404DF
:1039A7007515008A828B838CF012508FE582858390
:1039B700F045F06012D29090012C124FC3C2909044
:1039C700012C124FC3806B75C983806690F7F1E0B5
:1039D700FCBC015674022DFDE43EFE8D828E838F62
:1039E700F01257D7FDA31257D7FE90DE0EE4F090E2
:1039F700DE16E0FF7C007513088F828C83C007C03A
:103A070006C005C00412500FD004D005D006D00759
:103A1700EF4C601690DE20E0FB8D828E83F0A3AD25
:103A270082AE831FBFFF011C80E690F7DAE054FDEA
:103A3700FFF09000002290F7ECE0FF30E10A90FCE5
:103A4700667405F090FFFF2290DE0E7405F090DE9D
:103A570016E0FF8F4B754C0090DE17E0FCE4254B1A
:103A6700F54BEC354CF54C90F7EAE0FCA3E0FD4C48
:103A7700705890F7E6E4F0A3F090DE2AE090F7E8BC
:103A8700F090DE2AE090F7E9F090DE2AE0FD7C0076
:103A970090F7EAEDF0ECA3F090DE2AE0FAE4FB2DD4
:103AA700FDEA3CFC90F7EAEDF0ECA3F0E54B24FCD3
:103AB700F54BE54C34FFF54CC374049D74029C50E0
:103AC7000990F7EA7404F003A3F0E52955D16012D1
:103AD700D290900014124FC3C290900014124FC39B
:103AE70080E890F7E3E0FBA3E0FCA3E090F7E6E0D3
:103AF700FAA3E0FFEA2BFBEF3CFC7480252942D6B2
:103B070085268285278374DEF0852682852783A311
:103B1700742AF0852682852783A3A38C07EFF08577
:103B27002682852783A3A3A3EBF085268285278397
:103B3700A3A3A3A3A3A3A3E0543FF08526828527CD
:103B470083A3A3A3A3A3A3A3E054CF4410F07405B6
:103B57002526FEE43527FF90DE16E0FD8E828F8353
:103B6700EDF074042526FEE43527FF90DE17E08E7E
:103B7700828F83541FF5F0E054E045F0F090F7E6AC
:103B8700E0FEA3E0FFEE254BFCEF354CFDC37404CC
:103B97009C74029D500B7404C39EF54B74029FF5F1
:103BA7004CC37440954BE4954C502890FC667406C2
:103BB700F090DE14E0FD74FE5DF0751304900005CF
:103BC70012500F751310854B82854C8312500F903E
:103BD700FFFE22E52942D6E52942D7E54B2EFEE531
:103BE7004C3FFF90F7E6EEF0EFA3F0E52955D160E3
:103BF700FAE529F452D190F7E6E0FEA3E0FF90F74B
:103C0700EAE0FCA3E0FDC3EE9CEF9D402C90F7ECAF
:103C1700E04402F090F7EAE4F0A3F090DE0E7405BA
:103C2700F0AE2374BF5524FF8E238F2490DE14E05B
:103C3700FF74FE5FF09000012290DE0E7405F0AE77
:103C47002374BF5524FF8E238F2490DE14E0FF7466
:103C5700FE5FF09000002290F7ECE0FF20E10122E8
:103C670090F7E3E0FDA3E0FEA3E0FF90F807EDF097
:103C7700EEA3F090F7E8E0F55474FFB55402800323
:103C87000240F090F7E9E0FBBB800050030240D20E
:103C9700EB246F50030240D2EB2480FA240A83F509
:103CA70082EA241583F583E473D267FD3A1A5172C9
:103CB70089C2ABD2D2D2D22A5DB93C3D3E3F3E3F0C
:103CC7003F3F3F3F404040404040408D828E838F82
:103CD700F01257D7FA74012DF54FE43EF5508A528A
:103CE70075530090F7EAE552F0E553A3F0854F824C
:103CF700855083E0F5517401254FF554E43550F5AF
:103D070055A9518902E4F92552F552EA3553F5537D
:103D170090F7EAE552F0E553A3F085548285558381
:103D2700E0F8854F82855083A3A3884D894EE0FA3A
:103D3700E4254DF54DEA354EF54E854D35854E3624
:103D470090F7E8E0FA90F7E9E0F5328552338553CA
:103D5700348A82122E3790F7EAE4F0A3F00240E8A3
:103D67008D828E838FF01257D7FA8D828E83A38A26
:103D77004D754E00E0FA74022DF554E43EF5558A70
:103D8700018902E4254DF54DEA354EF54EA84DAAB9
:103D97004E90F7EEE8F0EAA3F090F7E6E0F9A3E03B
:103DA700FAE924FEF54DEA34FFF54E854D52854E6E
:103DB70053E5524553603D90F7EEE0F54FA3E0F52C
:103DC700507401254FF9E43550FA90F7EEE9F0EA1F
:103DD700A3F0855482855583E0FAA38582548583B1
:103DE70055854F82855083EAF0155274FFB552020C
:103DF700155380BD90F7E8E0FA90F7E9E0F53275E2
:103E070035EA7536F77533027534008A82122E3714
:103E17000240E890F7ECE0FA20E23C8D828E838F37
:103E2700F01257D7FA8D828E83A38A4D754E00E024
:103E3700FA90F80774022DF0E43EA3F08A01890294
:103E4700E4F9254DF54DEA354EF54EA84DAA4E90AD
:103E5700F7EEE8F0EAA3F090F7EAE0F9A3E0FA89D1
:103E67004D8A4EC37440954DE4954E5006754D40AE
:103E7700754E00E9C3954DF9EA954EFA90F7EAE9D0
:103E8700F0EAA3F090F807E0F552A3E0F553854D6B
:103E970054854E55E5544555603D90F7EEE0F54F96
:103EA700A3E0F5507401254FF9E43550FA90F7EE89
:103EB700E9F0EAA3F0855282855383E0FAA385826D
:103EC70052858353854F82855083EAF0155474FFDA
:103ED700B55402155580BD90F7E8E0FA90F7E9E090
:103EE700F5327535EA7536F77533027534008A820F
:103EF700122E370240E8D290900002C007C006C0D9
:103F070005124FC3C290900002124FC3D005D006CE
:103F1700D00790F7E8E0FA90F7E9E0F53290F7E696
:103F2700E0F533A3E0F5348D358E368A82122E37CD
:103F37000240E875350675365A8B3275330D753480
:103F470000855482122E370240E890FC67E0F8A300
:103F5700E0F9A3E0A3E0883589368B327533047521
:103F67003400855482122E370240E87535EE7536D7
:103F7700598B3275330E753400855482122E3702F1
:103F870040E890F7E6E0F533A3E0F5348B328D3562
:103F97008E36855482122E379000C8124FC31244B2
:103FA700B70240E87535E57536598B3275330975B3
:103FB7003400855482122E370240E88D828E838F1B
:103FC700F01257D7FC74012DF9E43EFABC020280C7
:103FD7000ABC03028021BC0429800DC002C0011263
:103FE7004580D001D002801AC290C002C00112459C
:103FF700CAD001D002800BC002C0011245A1D00176
:10400700D00290F7E8E0FC90F7E9E0F53290F7E6A8
:10401700E0F533A3E0F53489358A368C82122E37E2
:104027000240E890F7EA7401F0E4A3F075353675BD
:1040370036DF90F7E8E0FC90F7E9E0F53290F7EA31
:10404700E0F533A3E0F5348C82122E3790F7EAE4DB
:10405700F0A3F00240E88D028E048C017C0090FCF6
:104067006B7414F0745AA3F07480A3F07514098C60
:10407700158A8289838CF0C007C006C00512508F4D
:10408700E5828583F0D005D006D00745F0705275DC
:10409700C98090F7E8E0FC90F7E9E0F53290F7E6A1
:1040A700E0F533A3E0F5348D358E368C82122E374A
:1040B700802F90FC65E4F090FC66F090F809EDF035
:1040C700EEA3F0758202124118801690F7E6E0F52C
:1040D70033A3E0F5348B328D358E36855482122E1C
:1040E7003790F7ECE054FDF022E530453160198553
:1040F7003082853183121489AE82AF83EE4F701000
:1041070090F7ECE054FDF02290F7ECE054FDFFF05F
:1041170022E58290F80BF090F7ECE054FDF090F771
:10412700E8E0FF90F7E9E0F53290F80BE0FE8E3318
:1041370075340090F809E0F535A3E0F5368F820273
:104147002E37E52330E01175220274FE5523FEAFAA
:10415700248E238F2443BE01E5235406602F90FC51
:1041670065740AF075220374FD5523FEAF248E2370
:104177008F2490DE01E0FF74044FF0900008124F87
:10418700C390DE01E0FF74FB5FF075220190DE0E45
:10419700E4F090DE11E0FF30E21A90DE11E0FF74E8
:1041A700DB5FF090F7CFE4F0A3F090F7D4F0A3F043
:1041B70090F7DBF090DE0E7405F090DE11E0FF3033
:1041C700E52090DE11E0FF74CF5FF090FC66740885
:1041D700F090F7E1E4F0A3F090F7E6F0A3F090F7A2
:1041E700EDF090DE14E0FF30E62090DE14E0FF747F
:1041F7009F5FF090FC667408F090F7E1E4F0A3F09D
:1042070090F7E6F0A3F090F7EDF0E52320E20574D0
:1042170004B52214122F8C90FC65740BF074FB55B7
:1042270023FEAF248E238F24E52330E41112352299
:1042370074E75523FE740F5524FF8E238F24E5243E
:1042470030E65490FC65740CF0123A3DAE82AF83B1
:10425700BEFE41BFFF3E90F80C7406F0E4A3F09059
:10426700F7E8E0FF90F7E9E0F53275350C7536F8B9
:104277007533027534008F82122E3790F7E8E0FF0E
:1042870075350C7536F87532017533027534008F44
:1042970082122E37123C5EE52354E07006E5245463
:1042A700BD602990FC667409F075130890004412EC
:1042B700500F85238285248375131012500F741FA6
:1042C7005523FE74425524FF8E238F2422C0E0C05D
:1042D70082C083C007C006C005C004C0D075D00027
:1042E700E5BE30E6FB90DE06E0FF7E00E5234207F1
:1042F700E52442068F238E2490DE02E0FDE4CDC440
:10430700CD6DCD54F0CD6DFCED4207EC42068F2309
:104317008E2490DE04E025E0FCE4FD4207EC420633
:104327008F23EEF52430E11290F7ECE054FEF0AE67
:104337002374FD5524FF8E238F24758B00C2E8D08C
:10434700D0D004D005D006D007D083D082D0E032B9
:10435700C0E0C007C0D075D000E5BE30E6FBC2AFF5
:10436700E58930E703752203AFBE74FC5FF5BE75C0
:0E4377008900C2C5D2AFD0D0D007D0E032222C
:1059E5005344434376333530004348524F4E4F536B
:1059F5002072303435300000000000005253544E00
:105A050000554E494D504C454D454E544544005268
:105A1500455345545F4E4F570012011001000000D9
:105A250040501D47600001010203010A06100100F4
:105A350000004001000902200001010080FA09046C
:105A4500000002000001000705850240000107056E
:105A55000502400001040309040C035200660043DB
:105A650000610074001E034300680072006F006E41
:105A7500006F007300200044006F006E0067006C2B
:0F5A85000065000A03300030003900330000FFD5
:10438500AF83E58290F80EF0EFA3F090F80EE0FE13
:10439500A3E0FF7C007D008E028F038A828B83E081
:1043A500F9A3AA82AB83E960070CBC00EE0D80EB94
:1043B5007532F08C338D348E358F367582FE022E34
:1043C50037AF83E58290F810F0EFA3F090F810E096
:1043D500FEA3E0FF7C007D008E028F038A828B8323
:1043E500E493F9A3AA82AB83E960070CBC00ED0D49
:1043F50080EA8E358F367532F08C338D347582FEBA
:10440500022E37E58290F812F07535127536F8757B
:1044150032F17533017534007582FE022E37AF8394
:10442500E58290F813F0EFA3F07535137536F8753E
:1044350032F27533027534007582FE022E37AF8273
:10444500AE83ADF0FC90F815EFF0EEA3F0EDA3F020
:10445500ECA3F07535157536F87532F375330475BB
:0844650034007582FE022E37BF
:0514E400E4F50DF50E1A
:10446D007E197FF88FD57E197FF88ED47E217FF847
:10447D008FD37E217FF87F008ED28F147515188F04
:10448D001690F81975F0000255807403B50D06E409
:10449D00B50E02800280047582FF22AE0DAF0E05AF
:1044AD000DE4B50D02050E8E822290DF46E0FFBFB2
:1044BD00F00E90DF47E0FFBF0D0690DF487469F006
:1044CD00C2AF759A0075B80075A8001230E2AFBE84
:1044DD00747F5FF5BE75D69FC29002000022125503
:1044ED00F4AC82AD83AEF0FFC004C005C006C007BA
:1044FD009037BD75F086743D12547CAC82AD83AEA1
:10450D00F0FFE58124FCF581E4C0E0C0E074C0C09B
:10451D00E07441C0E08C828D838EF0EF125714ACA5
:10452D0082AD83AEF0FFE58124FCF5818C828D8315
:10453D008EF0EF125607AC82AD83AEF090DF09EE30
:10454D00F08D0390DF0AEBF090DF0BECF02275E1BC
:10455D000490DF3BE0FFBF01F890FC3CE0F5E190FB
:10456D00FC3CE0FFBF04012290DF3BE0FFBF0102F6
:10457D0080ED2290FC3CE0FFBF02012290DF13E0B2
:10458D00FF74F05FF0E0FF740F4FF090FC3C74028D
:10459D00F00249BF90FC3CE0FFBF03012290DF1306
:1045AD00E0FF74F05FF0E0FF740A4FF090FC3C7494
:1045BD0003F0F5E190DF3BE0FFBF13F82290FC3CE8
:1045CD00E0FFBF04012290DF13E0FF74F05FF0AF56
:1045DD009174EF5FF59175E10490DF3BE0FFBF0152
:1045ED00F8AF9B74FC5FF59BAFE974EF5FF5E99055
:1045FD00FC3C7404F02290FC3FE4F0A3F090FC32FC
:10460D00F0A3F090FC34F0A3F053C6C7759D008560
:10461D009E9E439E0485A9A943B90190FC3C740458
:10462D00F0751400751500F51690F83275F000123E
:10463D005580122CE7D2A87591D175E900750F0040
:10464D00439A0175E10490DF3BE0FFBF01F8227E44
:10465D00007F00C3EE94DCEF9405502490DF3CE026
:10466D00FD5450600490000122900032C007C00636
:10467D00124FF1D006D00774322EFEE43FFF80D3E7
:10468D0090000022AF83E58290FC5CF0EFA3F090E8
:10469D00FC5EE4F090DF02E0FF90DF3BE0FEBE1336
:1046AD000BB290C007124149D00780EDC29090FC2B
:1046BD00AAE4F090FC58E0FDA3E0FE90FCA0EDF024
:1046CD00EEA3F090FC5AE0FBA3E0FC90FCA6EBF00F
:1046DD00ECA3F090FC56E0F9A3E0FA90FCA2E9F00F
:1046ED00EAA3F090FCA4E9C39BF0EA9CA3F090FC34
:1046FD00A4E0FBA3E0FC8D148E158B828C83C00788
:10470D00C006C005C002C00112565BAB82AC83D09F
:10471D0001D002D005D006D00790FCA8EB29F0EC13
:10472D003AA3F0E94A705D90FC5CE0FBA3E0FC8BE2
:10473D00828C83E0F8881075110090FC56E510F01E
:10474D00E511A3F090DF04E0F8530003B8000280F8
:10475D0018B80102800302482390FC5674012510FD
:10476D00F0E43511A3F002482390FC5C74012BF0AA
:10477D00E43CA3F090FC56E0FBA3E0FC90DF02EBE1
:10478D00F002482390DF04E0FC530403BC000280D8
:10479D0046BC0102800302482390FC5CE0FBA3E0D1
:1047AD00FC90FC5FE9F0EAA3F090FC617401F0E489
:1047BD00A3F08B828C83C007C002C001124F6ED054
:1047CD0001D002D00790FC5CE0FBA3E0FC89008BDC
:1047DD00828C83E8F0803FED4E603690FCA8E0FDC2
:1047ED00A3E090DF02EDF090DF04E0FE74FC5EF0DC
:1047FD0090FCA8E0FDA3E0FEC374FF9DE49E50096C
:10480D0090DF04E0FE74024EF090FCAA7401F0807B
:10481D000590DF02E9F0D2A890FCABE0FE20E303A7
:10482D0002495190DF04E0FE530603BE010690FCE1
:10483D005E7401F090FC5EE0FE90FC5CE0FCA3E099
:10484D00FDEE2CFAE43DFB90FC56E0F8A3E0F99068
:10485D00FC7DE8F0E9A3F08A828B83C007C006C017
:10486D0005C0041252BDAA82AB83D004D005D00678
:10487D00D00790FCABE0F9530104B90448C007EE32
:10488D002CF8E43DF990FCABE0FF5307F090FC8170
:10489D00E8F0E9A3F090FC83EAF0EBA3F090FC853F
:1048AD00EFF088828983C007C006C005C004C0032D
:1048BD00C0021252F7D002D003D004D005D006D0DA
:1048CD0007D0078046C007EE2CF8E43DF990FCAB0D
:1048DD00E0FF5307F090FC88E8F0E9A3F090FC8A24
:1048ED00EAF0EBA3F090FC8CEFF088828983C0078F
:1048FD00C006C005C004C003C002125340D002D090
:10490D0003D004D005D006D007D007EE601E90FC72
:10491D00ABE0FE5306F0BE50098C828D837410F00F
:10492D0080228A068C828D83EEF0801890FCABE09D
:10493D00FE5306F0BE500890DF027410F080059013
:10494D00DF02EAF090FC5CE0FDA3E0FE90FC38EDA8
:10495D00F0EEA3F090FC9EE4F0A3F075E1037D6012
:10496D007EEA90DF3BE0FCBC1302801C1DBDFF0105
:10497D001EED4E6013B290C007C006C0051241492E
:10498D00D005D006D00780DAD290ED4E700690FC9F
:10499D00667413F090DF3BE0FEBE130BB290C007C0
:1049AD00124149D00780EDC29090DF02EFF0758281
:1049BD000122D2A875140075150075160290F832F3
:1049CD0075F00012558090FC32E4F0A3F090FC34A9
:1049DD00F0A3F090FC36F090FC3704F090F831E441
:1049ED00F0AF9B74FC5FF59BAFE974EF5FF5E97574
:1049FD00E10290DF3BE0FFBF0DF84391102290FCE8
:104A0D00AD7401F02290FCADE4F022C021C0E0C0F5
:104A1D00F0C082C083C007C006C005C004C003C07B
:104A2D0002C001C000C0D075D00090FC657411F0BB
:104A3D00C28990DF3BE0FFBF0D028003024B62D2C3
:104A4D009090FC97E0E0602A90FC98E0FEA3E0FFD8
:104A5D0090FC98E024FFFCA3E034FFFD90FC98EC63
:104A6D00F0EDA3F074FF2F400990DF04E0FF74FC1C
:104A7D005FF090FC3C7402F090F831E025E0FEE42C
:104A8D002432FFEE34F8FEE075F002A42432FC74FB
:104A9D00FC35F0FD8C828D83E0FAA3E0FB74012AD6
:104AAD00F8E43BF98C828D83E8F0E9A3F0EA2FF569
:104ABD0082EB3EF583E5D9F090F831E075F002A474
:104ACD002432F58274FC35F0F583E0FEA3E0FFC3DC
:104ADD009402501A90F831E075F002A42432F58258
:104AED0074FC35F0F583E0FEA3E0FF4E701A90F8EC
:104AFD0031E0FF75F002A42432F58274FC35F0F537
:104B0D008374FFF07401A3F090FC98E0A3E090FC97
:104B1D0098E0F5F0A3E045F06003024D1F90FC977F
:104B2D00E0E07003024D1F90FC9AE0FEA3E0FF90C1
:104B3D00FC98EEF0EFA3F090FC98E0FEA3E090DF80
:104B4D0002EEF090DF04E0FF74FC5FF0E0FF740212
:104B5D004FF0024D1F90DF3BE0FFBF1302800302B9
:104B6D004D1F90FCAAE0E07003024CB090FC4EE0AB
:104B7D00FEA3E0FF0EBE00010F90FC4EEEF0EFA382
:104B8D00F090FC9EE0FEA3E0FF90FCA2E0FCA3E011
:104B9D00FDEEB50406EFB505028003024C8390FCD3
:104BAD00A0E0A3E090FCA0E0F5F0A3E045F06037B5
:104BBD0090FCA0E0FEA3E0FFBEFF05BF0002801445
:104BCD0090FCA0E024FFFEA3E034FFFF90FCA0EEDC
:104BDD00F0EFA3F090FCA6E0FEA3E0FF90FC9EEEAC
:104BED00F0EFA3F0024C8390FCA2E0F514A3E0F5E6
:104BFD001590FC9CE0FF7E008F828E8312565BAE7B
:104C0D0082AF8390FC38E0FCA3E0FDEE2CF582EF43
:104C1D003DF583E4F090FC9CE02401F0E0FF90FC76
:104C2D009DE0FEEFB5060590FC9CE4F090FCA2E043
:104C3D00F514A3E0F51590FC9CE0FF7E008F828EAD
:104C4D008312565BAE82AF8390FC38E0FCA3E0FD8F
:104C5D00EE2CFEEF3DFF8E828F83E0701090FC41B5
:104C6D00E4F090FC667412F012455BC29090FC9ECD
:104C7D007401F0E4A3F090FCA8E0FEA3E0FF90FC2B
:104C8D00A8E024FFFCA3E034FFFD90FCA8ECF0EDC0
:104C9D00A3F0BEFF22BF001F90DF04E0FF74FC5F96
:104CAD00F0801490FCA8E024FFFEA3E034FFFF90F9
:104CBD00FCA8EEF0EFA3F090FC3C7403F090FCA286
:104CCD00E0F514A3E0F51590FC9CE0FF7E008F82CB
:104CDD008E8312565BAE82AF8390FC9EE0FCA3E008
:104CED00FD90FC9EE02401F0A3E03400F0EC2EFEDC
:104CFD00ED3FFF90FC38E0FCA3E0FDEE2CF582EFDC
:104D0D003DF583E0F5D990FC3AE02401F0A3E034C1
:104D1D0000F0D0D0D000D001D002D003D004D00507
:104D2D00D006D007D083D082D0F0D0E0D02132C0D1
:104D3D0021C0E0C0F0C082C083C007C006C005C05E
:104D4D0004C003C002C001C000C0D075D0007512F0
:104D5D000090FC657410F0AE9B74FC5EF59BE5E96C
:104D6D00420FE5E930E02090FC3DE0FDA3E08D062B
:104D7D007D00AB9C7C0090FC3FED4BF0EE4CA3F026
:104D8D00AEE974FE5EF5E9E5E954707003024F1F5C
:104D9D0090FC3CE0FEBE030AAE0F748F5EF50F0271
:104DAD004F1890F831E0FEB40100E4332436F5825B
:104DBD00E434FCF583E0FEBE01028003024EF59063
:104DCD00FCABE0FE20E103024ECE90DF04E0FE538B
:104DDD000603BE010375120190FCABE0FE53060104
:104DED00BE017090F831E025E0FDE42432FEED3493
:104DFD00F8FDAB127C00EB2EFEEC3DFDE0F929FA3F
:104E0D00E42432F9EA34F8FAEB29FBEC3AFCE075CC
:104E1D00F002A42432F58274FC35F0F583E0F9A399
:104E2D00E0FAA8127F00E9C398F9EA9FFA90FCAB6B
:104E3D00E0FF5307F090FC81EBF0ECA3F090FC83C6
:104E4D00E9F0EAA3F090FC85EFF08E828D8312528B
:104E5D00F7806E90F831E025E0FEE42432FFEE3469
:104E6D00F8FEAC127D00EC2FFFED3EFEE025E0FAE2
:104E7D00E42432FBEA34F8FAEC2BFCED3AFDE07554
:104E8D00F002A42432F58274FC35F0F583E0FAA328
:104E9D00E0FBA8127900EAC398FAEB99FB90FCAB02
:104EAD00E0F95301F090FC88ECF0EDA3F090FC8A52
:104EBD00EAF0EBA3F090FC8CE9F08F828E83125315
:104ECD004090F831E0FF74016FF0E0FF75F002A43F
:104EDD002432F58274FC35F0F583E4F0A3F090FCF8
:104EED0036F090FC37F0802190FC667412F0B29091
:104EFD0090F831E0FF75F002A42432F58274FC3590
:104F0D00F0F583E4F0A3F0B290C290AFE974CF5FF7
:104F1D00F5E9E5E930E61490FC667410F0B29012F4
:104F2D00455BB290AFE974BF5FF5E9E5E930E71491
:104F3D0090FC667411F0B29012455BB290AFE974BB
:104F4D007F5FF5E9D0D0D000D001D002D003D004DE
:104F5D00D005D006D007D083D082D0F0D0E0D021BC
:104F6D0032AF83E58290FC63F0EFA3F090FC61E03B
:104F7D00FEA3E0FF90FC63E0FCA3E0FD90FC5FE08E
:104F8D00FAA3E0FB8A008B011ABAFF011BE8496006
:104F9D0024EE2AF8EF3BF9E82CF8E93DF9EA2CF577
:104FAD0082EB3DF583C006C007E088828983F0D08F
:064FBD0007D00680CF22A0
:105A94000000000000000100000000000000000001
:075AA40000000000000000FB
:104FC300AE82AF831EBEFF011FC3E49E74808FF0C9
:104FD30063F08095F050167C4C7D04EC24FFFAEDD1
:104FE30034FFFB8A048B05EA4B70F080D722AE8234
:104FF300E583CE25E0CE33FF1EBEFF011FC3E49E33
:1050030074808FF063F08095F040ED22AE82AF8321
:10501300D2909003E8C007C006124FC3C29090011C
:10502300F4124FC3D006D0071513AD13ED20E75488
:10503300EE30E024900019C007C006C005124FC32C
:10504300D290900226124FC3C290900019124FC300
:10505300D005D006D0078022900113C007C006C038
:1050630005124FC3D290900032124FC3C2909001E9
:1050730013124FC3D005D006D007EFC313CE13CE00
:10508300FF1D80A8C2909003E8024FC3AFF0AE8328
:10509300E58290FC6EF0EEA3F0EFA3F090FC6EE0DF
:1050A300FDA3E0FEA3E0FF90FC6BE0FAA3E0FBA30B
:1050B300E0FCA814A915E8496050C000C0018D8226
:1050C3008E838FF01257D7F98A828B838CF0125715
:1050D300D7F8E9C398F98916D001D0006010E51616
:1050E300F5173395E0F518851782851883220DBDD2
:1050F30000010E90FC6EEDF0EEA3F0EFA3F00ABA00
:1051030000010B18B8FF011980AC90000022AFBE5C
:1051130074FB5FF5BEE5BE30E6FBAFC674B85FF562
:10512300C6E5C620E6FB43BE04E5BE30E6FB53C638
:10513300C743E40C43E401D2B92243FE03C29022E5
:10514300C0E0C082C083C0D090FC67E02401F0A31C
:10515300E03400F0A3E03400F0A3E03400F0D0D05A
:10516300D083D082D0E032124497AF8290FC75EFA7
:10517300F08FF005F07401800225E0D5F0FB90FC80
:1051830076F0EF75F008A42419FE74F835F0FF905B
:10519300FC71EEF0EFA3F08E828F83A3A374DFF094
:1051A3008E828F83A3A3A374B1F08E828F83A3A374
:1051B300A3A3A37410F074062EF582E43FF583E0F5
:1051C30054E0441DF074072EF582E43FF583E05468
:1051D3003F4440F074072EF582E43FF583E054FC2E
:1051E3004401F0124497AF8290FC77EFF08FF00503
:1051F300F07401800225E0D5F0FB90FC78F0EF75A8
:10520300F008A42419FE74F835F0FF90FC73EEF057
:10521300EFA3F08E828F8374DFF08E828F83A3746B
:10522300B2F08E828F83A3A3A3A3A37410F074069A
:105233002EF582E43FF583E054E0441EF074072E1C
:10524300F582E43FF583E054CF4410F074072EF564
:1052530082E43FF583E054FC4401F043A91043B9D1
:105263001022AF83E58290FC7BF0EFA3F0E5B3302F
:10527300E3FB90FC71E0FEA3E0FF90FC7BE0FCA36A
:10528300E0FD8C028D038B028E828F83EAF090FC0B
:1052930071E0FEA3E0FF8E828F83A37D00ECF0908C
:1052A300FC76E042D690FC79E0FF90FC7AE0FE4F7A
:1052B3004401F5B3E5B330E3FB22AF83E58290FC11
:1052C3007FF0EFA3F090FC7FE0FEA3E0FF90FC7D76
:1052D300E0FCA3E0FDEC540F60158C028D030CBCC5
:1052E30000010DEA2EF582EB3FF583E4F080E68CB6
:1052F300828D8322AF83E58290FC86F0EFA3F0904A
:10530300FC86E0FEA3E0FF90FC81E0FCA3E0FD90BF
:10531300FC83E0FAA3E0FB90FC85E0F990FC8FECC2
:10532300F0EDA3F090FC91EAF0EBA3F090FC93E492
:10533300F090FC94E9F08E828F8302538AAF83E569
:105343008290FC8DF0EFA3F090FC8DE0FEA3E0FFD4
:1053530090FC88E0FCA3E0FD90FC8AE0FAA3E0FB6C
:1053630090FC8CE0F990FC8FECF0EDA3F090FC91B5
:10537300EAF0EBA3F090FC937402F090FC94E9F054
:105383008E828F8302538AAF83E58290FC95F0EF80
:10539300A3F0E5B330E3FB90FC95E0FEA3E0FF90C0
:1053A300FC8FE0F51AA3E0F51B90FC94E0FB74502E
:1053B3005BF51990FC93E0F94B4401FB740149F54B
:1053C3001890FC91E0F514A3E0F515E4F516F51734
:1053D300C3E5169514E5179515400122C00390FC0B
:1053E30071E0F8A3E0FBE5162EF9E5173FFA89040F
:1053F3008A058D0488828B83ECF090FC71E0FCA31A
:10540300E0FD8C828D83A3E9F090FC73E0FCA3E0C4
:10541300FD8C828D83A3A3E516251AFCE517351BA6
:10542300FD8C028D038B02EAF090FC73E0FAA3E09B
:10543300FB8A828B83A3A3A3ECF090FC78E0FD901E
:10544300FC76E0FC4D42D6D003E5196017E5142441
:10545300F0FCE51534FFFDECB51609EDB517058530
:1054630018B380028BB3E5B330E3FB74102516F554
:1054730016E43517F5170253D312551FBC00030268
:1054830056E6EF60FA30D502B2D1E583B4FF0302EA
:1054930056FCE582B4FF030256FC258340072482B1
:1054A300400B0256E624831450030256FCF582EAAD
:1054B3008DF0A4A8F0EA8EF0A428F8E435F0F9EB17
:1054C3008DF0A428E935F0F9E433CA8FF0A429F963
:1054D300EA35F0FAEBF88EF0A429F9EA35F0FAE4AC
:1054E30033FBEC8DF0A429F9EA35F0FAE43BFBE851
:1054F3008FF0A42AFAEB35F0FBE433CCFD8EF0A455
:105503002AFAEB35F0FBE43CFCED8FF0A42BFBEC2B
:1055130035F0FC20E70312554D0256C5AA82AB8332
:10552300A2F73392D1F5826002D2F7ACF0E5812481
:10553300F9F8E6FD08E6FE0886F008E6A2F73392DE
:0A554300D5F5836002D2F7AFF02225
:0614BA00E478FFF6D8FD06
:10554D007804EC7011E58224F8500AF582E4C9CA9A
:10555D00CBFCD8EF22EC7820058220E713D5820111
:10556D0022C3E933F9EA33FAEB33FBEC33FCD8EA27
:10557D00158222AC82AD83AE15AF16BE0004EF606E
:10558D000C1F0FE514125640A3DEFADFF88C828D46
:10559D008322AD82AE83AFF08D198E1A8F1B8514C9
:1055AD001C85151D85161EA817A9188803890418B2
:1055BD00B8FF0119EB4C6025851C82851D83851E66
:1055CD00F01257D7FCA385821C85831D8D828E8397
:1055DD008FF0EC125640A3AD82AE8380CE8519823A
:0755ED00851A83851BF022E3
:101498007917E94400601B7A01905A9478977593FC
:1014A800FCE493F2A308B800020593D9F4DAF275C4
:0214B80093FFA0
:1055F400FCABF0AA83A982749EC2D1F58212554DE8
:105604000256C57F9E12562E30D1030256E6C3EFD2
:105614009582500974FFF5F0F583F5822279001222
:1056240057F389828A838BF0EC22AA82AB83A2F798
:105634003392D1F5826002D2F7ACF02220F7113018
:10564400F6138883A88220F509F6A88375830022BF
:1056540080FEF280F5F022E5828514F0A4C582C0B4
:10566400F08515F0A4D0F025F0C5838514F0A425A9
:1056740083F58322E514451560467A01E51425E097
:10568400F514E515334012F515E5829514E5839577
:105694001540030A80E6C3E51513F515E51413F563
:1056A40014C3E5829514F5F0E58395154005F5835B
:1056B40085F082C3E51513F515E51413F514DAE145
:0156C40022C3
:1014C0007800E84400600A79007593F0E4F309D8E5
:1014D000FC7897E8440C600C790D90F000E4F0A3E0
:0414E000D8FCD9FA61
:02148900E4730A
:1056C500B98003EA13B34010EA2401FAE43BFBE492
:1056D5003CFC50047C800582BC000EBB000BBA006C
:1056E50008E4F5F0F583F58222A2D1E582138CF06A
:1056F50092F78B838A8222E4F583F58275F080F434
:10570500A2D11322E4F583F58275F0C0747F2212CD
:10571500551F30D502B2D1BF0009BC00030257099D
:105725000256FCBC00030256E6E583B4FF0BE58296
:10573500B4FF030257090256E6E582B4FF03025699
:10574500FCC395835007247F400B0256E624801442
:1057550050030256FCF582C3ED9AEE9BEF9C401177
:105765001582C3EA33F9EB33FAEC33FBE433FC80FF
:1057750005E4CCCBCAF9C08275F019C3E99DEA9E50
:10578500EB9FEC9400D5F002802D400EE99DF9EADF
:105795009EFAEB9FFBEC9400FCC3B3E833F8E5827B
:1057A50033F582E58333F583C3E933F9EA33FAEB5D
:1057B50033FBEC33FC80C4B3E4F938FAE43582FBFF
:1057C500E43583FCD082500405827C8012554D025D
:0257D50056DD9F
:0D148B00758155125836E582600302148603
:1057D70020F71430F6148883A88220F507E6A883FB
:1057E70075830022E280F7E49322E0226040F825E7
:1057F70082500274FFF582E824F8501ECCCBCAF918
:10580700E4CC24F85014CBCAF9E4CB24F8500BCAE3
:10581700F9E4CA24F8500379002224086010F8C379
:10582700EC13FCEB13FBEA13FAE913F9D8F1227531
:03583700820022CA
:00000001FF
